:020000020000FC
:1000000003C0189518950EC00FE107BB00E008BBB0
:1000100000E808B905E003BF0CEC02BF02E009BF2D
:1000200078943DC01FB72CEC22BF1FBF189502E289
:1000300005BF00E40BBF789488950895436F7079ED
:10004000726967687473207265736572766564207F
:100050004469636B2043617070656C7320777777B8
:100060002E70726F6A656374732E63617070656C55
:10007000732E6F7267204F63746F6265722032381F
:100080002C203230303820436F64653A20543132AE
:10009000617374726F626530383130323841C09AA2
:1000A000C19AC29AC39AC49AC2DFC198C398C4982D
:1000B000BEDFC098C198C298C49AB9DFC498B7DFB0
:1000C000C49AB5DFC39AC09AC29AC498B0DFC398E5
:1000D000C49AADDFC098C298C498A9DFC49AA7DFBC
:1000E000C498A5DFC09AC19AC49AC29AC39A9FDFE6
:1000F000C198C398C4989BDFC098C198C298C49A0D
:1001000096DFC49894DFC49A92DFC09AC498C29ACA
:10011000C39A8DDFC398C49A8ADFC098C298C498E6
:0C01200086DFC49A84DFC49882DFB9CF68
:00000001FF
